:101800002DC046C045C044C043C042C041C040C0D6
:101810003FC03EC03DC03CC03BC03AC039C038C0EC
:1018200037C036C035C0E7C116C2FCC1AEC2ADC2BA
:1018300001C2ABC2AAC2A9C2A8C2A7C2A6C2A5C2FF
:10184000A4C2A3C208C207C201C22AC206C276C28B
:1018500059C29BC29AC299C28DC284C211241FBEB2
:10186000CFE5D4E0DEBFCDBF10E0A0E6B0E0ECE411
:10187000FEE102C005900D92A436B107D9F711E040
:10188000A4E6B0E001C01D92A63AB107E1F7ABC2F1
:10189000B7CF0F92AF93BF93CF93DF93EF93FF93A5
:1018A000FC01EA01DB01C895099231961197D9F73D
:1018B000FF91EF91DF91CF91BF91AF910F9008957C
:1018C0000F921F920F93AF93BF93CF93DF93EF933A
:1018D000FF93FC01EA01DB010990199001E043D07C
:1018E00032961297C9F7FC0103E03DD005E03BD0EA
:1018F000FF91EF91DF91CF91BF91AF910F911F9029
:101900000F9008950F931F93EF93FF93FC0103E053
:101910002AD000E410E0E00FF11FE617F707B9F74F
:10192000FF91EF911F910F9108950F930F9222D085
:10193000082E09E018D00F900F9108950F930F9281
:10194000EF93FF9317D0FC0160935700C895802D4B
:10195000FF91EF910F900F9108950F930BD001E13C
:1019600002D00F910895E199FECF00935700E895BA
:10197000FFFF00000091570000FDFCCF089583E0B9
:1019800089B98AB188618AB908958AB1877E8AB98E
:1019900008958CB95E9BFECF5E9A08958CB199270D
:1019A00008958BB19927807890700895EF92FF92F7
:1019B0000F931F93CF93DF937B01C0E0D0E0C61756
:1019C000D70760F48C01EDDF8823E9F3E7DFF80146
:1019D00081938F012196CE15DF05A8F381E090E079
:1019E000DF91CF911F910F91FF90EF900895EF92AB
:1019F000FF920F931F93CF93DF937C018B01C0E085
:101A0000D0E0C017D10730F4F70181917F01C1DF29
:101A10002196F7CF81E090E0DF91CF911F910F9158
:101A2000FF90EF900895EF92FF920F931F93CF9343
:101A3000DF937C0100E010E00817190780F4C0E094
:101A4000D0E00000AEDF882351F4219683E0CB364E
:101A5000D807B8F30F5F1F4F0E151F0580F3DF91F6
:101A6000CF911F910F91FF90EF9008958EDFDBDFF4
:101A70000895DF92EF92FF920F931F93CF93DF931E
:101A8000CDB7DEB72197DEBFCDBF8C017B011982B8
:101A9000D98061E070E0CE01860F971F87DF8981D2
:101AA0008B31B9F761E070E0C80180DF61E070E080
:101AB000CE01860F971F7ADF89819927182F00277B
:101AC00061E070E0CE01860F971F70DF8981080FFB
:101AD000111D61E070E0CE01860F971F67DF8981DD
:101AE0008E30B1F4C8010196BC01C7015FDF9801D7
:101AF0008FEF0F3F180779F0F70181917F01D8260A
:101B000021503040FFEF2F3F3F07B1F7DD2019F0A4
:101B100080E090E001C0C8012196DEBFCDBFDF911B
:101B2000CF911F910F91FF90EF90DF900895CF928A
:101B3000DF92FF920F931F93CF93DF93182FEB0148
:101B40006A018BE126DF4BE1F42E812F22DFF126A3
:101B50000D2F1127802F1DDFF0268C2F1ADFFC267A
:101B60008EE017DF8EE0F82621978FEFCF3FD80762
:101B700051F0F60181916F01F8260BDF2197FFEFFD
:101B8000CF3FDF07B1F78F2D04DFDF91CF911F919A
:101B90000F91FF90DF90CF9008959927813991059B
:101BA00059F08239910524F48039910529F008C053
:101BB0008239910519F004C082E003C087E001C0BA
:101BC00080EC99270895BF92CF92DF92EF92FF9217
:101BD0000F931F93CF93DF93B82EEB018881992742
:101BE000AA27BB27FC013197EB31F10508F0CDC0E6
:101BF000ED5EF34F0994198288E08A8381E48B8338
:101C000086E58C8382E58D8389E48E8383E58F83EB
:101C100080E588878FE5898782E38A87AB016BE05F
:101C200070E0B8C08981B9DF8A831982AE0163E0B0
:101C300070E0B0C08B819927982F88272C81820F64
:101C4000911D9093A5018093A40105C060E070E20E
:101C500080E090E057DE19829AC089819927182F79
:101C600000278A819927082B192B1982CB0102960C
:101C70002091A4013091A501AC01B801C901880FE0
:101C8000991F07DEFE01E00FF11F128298013695C1
:101C900027958091A4019091A501820F931F45C0C3
:101CA00089819927182F00278A819927082B192BBA
:101CB000CC24DD24C016D106D0F4FAE0EF2EF12CAE
:101CC000E60EF71E8091A4019091A501880F991F3F
:101CD000A70160E470E08C0D9D1DF2DD80E490E0D2
:101CE000C80ED91EE80EF91EC016D10658F335DE0F
:101CF0001982169507958091A4019091A501800FF6
:101D0000911F2BC089819927182F00278A81992735
:101D1000082B192B1982FE01E00FF11F128280910E
:101D2000A4019091A501800F911F9093A50180932C
:101D3000A4010D5F1F4FAE01B8012CC08981992706
:101D4000382F22278A819927282B392B19828091B5
:101D5000A4019091A501820F931F9093A5018093F8
:101D6000A40115C019828C81E82FFF27E05AFF4F8C
:101D7000808105C0198269E081E090E0DFDD8A831F
:101D80001B82AE0164E070E005C089EC8983AE017E
:101D900062E070E08B2DCBDEDF91CF911F910F9130
:101DA000FF90EF90DF90CF90BF900895CF93DF9397
:101DB000CDB7DEB72197DEBFCDBF69E081E090E00F
:101DC000BDDD992784FF07C08F7EAFDD04C064E6C8
:101DD00070E08981F8DE64E670E0CE01019649DEAC
:101DE000892BA9F3F8CFCFE5D4E0DEBFCDBFCEE19C
:101DF000F894AEEFB1E021D0802D843B61F4AFEFD9
:101E0000B1E01BD0802D833C31F4ADEFB1E015D0B3
:101E1000802D992781BFB3DDC1DD84E690E003DE2C
:101E2000C0DD882311F0C2DF04C0C150C8BBCC2381
:101E3000A1F71CDE80E090E008C0E199FECFBFBBB7
:0C1E4000AEBBE09A11960DB20895FFCFE2
:041E4C001E930700DA
:0400000300001800E1
:00000001FF
